:021B2B00EFF8D1
:061B0D00000000D8FB22DD
:061B1300F07814021B0D26
:10192000908000E521D2E0121B136403121B1364A4
:0B19300003121B13DFEFC2E0021B13C9
:10119200C243EE2F604A0ED3121970303A0090808B
:1011A20000E521203A05D2E0121B136403121B133F
:1011B2006403121B13203A05C2E0121B13EFBE0197
:1011C20005C3940440045CB40112C3121970A9301F
:1011D2007840121B0DD9F9DFBEDEBC22DFC3DEC1AF
:0711E200908002E523F022DA
:10185900EE2F601E0E908000E521D2E0121B13646A
:1018690003121B136403121B13C2E0121B13DFEADA
:03187900DEE82284
:1016FC00A243923FC243121134EE2F60140E90801D
:10170C0000E5216403121B136403121B13DFF4DEC8
:0B171C00F2121A3EC239A23F92432293
:101A3E00E523908002D2E4F07828121B0DC2E4F068
:051A4E007828021B0DC9
:1011340012113BC3021970D3121970908000E5217B
:10114400D2E1F07817121B0D204B25C2E0C2AFF09C
:10115400E523908002C2E0F0D2AF780C121B0DD2CE
:10116400E0C2AFF0908000E521D2E1F0D2AF80136D
:10117400E523908002D2E1F0780C121B0DC2E1F05D
:0E1184009080007812121B0DE521F0D2392266
:101A5300EF6011908000E5216403121B13640312ED
:051A63001B13DFF4225B
:0C1AED00908003E524C2E6F0D2E6F0226F
:10197000E5254004D2E68002C2E6908004F0F52519
:081980004001227805021B0D55
:100E3900907DC1E054F0B4F0061212A9020EBBB4C1
:100E49000005120D14806BB410051215D88063B417
:100E59002005121390805BB430051217ED8053B44E
:100E6900400512189E804BB45005120F378043B4C9
:100E79006005121A90803BB470051215A28033B434
:100E8900800512100E802BB49005120EC28023B477
:100E9900A005121AC2801BB4B00512152E8013B416
:100EA900C00512193B800BB4D00512193B800312FF
:090EB9000FA3907FC97400F02220
:051B1900740602193DF5
:051B1E00741502193DE1
:10193B007418C252753400901B4C858331858232EA
:0B194B00F0A37400F0F52C752D0122B4
:10187C00C252753400901B4C85833185823274A51D
:10188C00F0A3E516F0540F240354FE03F52D752C2C
:02189C00002228
:101A9000901B4E7462F5167402F0A37442F00218A3
:011AA0007CC9
:1012A900A3E0A3B403030213DEB40A030213DCB4FC
:1012B9000003021AA1B40403021751B40503021270
:1012C900F6B40603021343B40703021727B408054B
:1012D900E0FF021A7DB4090BE0FFA3E0FD12146AD6
:0D12E900021B19B40D0612113B021B192245
:101A7D00121672901B4E74F2F5167408F0A3EFF067
:031A8D0002187CC0
:101AA1001217A1E0F512FEA3E0F513FF050A021BD0
:011AB100191B
:1013DC00050A050A1217A1E0FEF512A3E0FFF513AA
:1013EC00C3E51D9420E51C9400500A204807E4B581
:1013FC000A0302193BD252907DC2E0B4030280036F
:10140C00B40A0F7C00907DC7E0FD14250AF50A1282
:07141C0010D48E2C8F2D224D
:101751007400F50AE51C451D601B30480F908000A0
:1017610078007900E030E104D8FAD9F8121AED7561
:081771001C00751D00021B198C
:1012F6001217A1E0FCA3E0FDA3E0F8A3E0F9A3E048
:10130600FAA3E0FB901B4BECF0E525D2E1D2E0BC62
:101316000306C2E0D2E18007BC0204C2E1D2E0F5D6
:1013260025908004F0901B48EDF0901B49E8F0A34F
:0D133600E9F0901B46EAF0A3EBF0021B1952
:10172700907DC6E0FEA3E0FF907DC3E0B4000D30DE
:101737003A051216FC8010121859800B3038051222
:0A1747001A288003121779021B19FB
:10134300907DC4E0FF7E00A3A3A3E0FCA3E0FD1215
:1013530010D4907DC3E0B40020303A08203905C290
:10136300431211347C07907DC1E0907DC9540FB4C2
:101373000802E0FC121192801130380B203D031259
:0D138300160C1217C88003121779021B19EF
:1017A100907DC3E0B40009204A19D24A7D408007E8
:1017B100304A10C24A7D207F1012146A7DD87F0002
:0717C10012146A907DC4229E
:100FA300A3E0A3C3B400028032B40102800BB402F5
:100FB300028029B40302800222D3121003907DC65B
:100FC300500CE584F8E0A3F608DFFA021B19E0A34E
:100FD3000586F0A30586DFF6021B19D312100390D2
:100FE3001B4E7516E8500CE584F8E608F0A3DFFA0B
:100FF30002187C0586E0A30586F0A3DFF602187CC1
:0B100300E0FFA3E0F584A3E0F58522E8
:1016A300907F98E0C2E3F0C2E5F0F879C77B027A55
:1016B30008E933F9E8C2E45002D2E4F0D2E3F0C21D
:0D16C300E3F0DAEDEFF9DBE7E8D2E5F02225
:10142300907F98E0C2E3F0C2E5F0FB79A77A08E980
:1014330033F9EBC2E45002D2E4F0D2E3F0C2E3F0BA
:10144300DAED7828000000D8FB7A087F00907F9BB4
:10145300E0C372E2EF33FF907F98EBD2E3F0C2E395
:07146300F0DAEAD2E5F02205
:10146A00C2AF907F98E0D2E3F0908003E524D2E403
:10147A00F0F524EFF9907F98E0F87B027A08E933D7
:10148A00F9E8C2E45002D2E4F0C2E3F0D2E3F0DABF
:10149A00EDEDF9DBE7908003E524C2E4F0F524D210
:0214AA00AF226F
:1014AC00C2AFE520907F97FA7809EAC2E6F0791E80
:1014BC00D9FEEAD2E6F0D3EF00007907D9FE33CAA1
:1014CC004008C2E6F0CAD8F28006D2E6F0CAD8EAE2
:1014DC00D2AF907F997A03E030E105D8FADAF8C3FD
:0114EC0022DD
:10167200907F96E020E0047E0180027E008E0CEFD7
:101682006009907F96E054FEF0800B907F96E044D4
:1016920001F0A23A9243E50C70047F0180027F00C0
:0116A2002225
:100D1400C246907DC5E0540CF50CE030E424907D8F
:100D2400C3E0F539A3E0F53CE53854F34404F53861
:100D3400D24CE50C7047C24CE53854F34408F538FE
:100D4400803B907DC2E0F50BA3E0F511A3E0F5171D
:100D5400E53854FC4401F538D24FE50C700AC24F13
:100D6400E53854FC4402F538A23A9243C251C24ECB
:100D7400303A0AAF14EF651460FB121A3EE50CB466
:100D84000403121640E50CB40803121568121B196B
:100D9400C2AF907DC5E030E706D23CD251D24EA21C
:060DA40051B39246D2AFEC
:010DAA002226
:1015D800C246907DC2E030E014E538540C602053D8
:1015E80038F3304C1A12156843380C8012E5385419
:1015F80003600C5338FC304F06121568433803D289
:0416080046021B1962
:10139000C2AF907DC2E030E407E0A2E3925B803709
:1013A000C25BC255907DC3E0901B5CF0907DC2E0B3
:1013B00030E10BA3E0F510E4901B43F08019907D21
:1013C000C2E030E00CD255907DC4E0901B43F08029
:0C13D00006901B437401F0D2AF021B1901
:1017ED00E4901B4EF030550204F0901B5CE0901B12
:1017FD004FF0A3E515F0A37480F0A3E53AF075164C
:04180D003502187C0C
:10189E00C2AF907DC2E0F50DA3E0F508A3E0F50E12
:1018AE00A3E0F509C253A3E030E002D253D2AF0257
:0218BE001B19F4
:100F3700121B19C2AF907DC2E0F50C7F02C28E90E2
:100F47007DC4E0F4F58B907DC3E0F4F58DE589541D
:100F57000F4410F58953883FC28FC206907F97E5EB
:100F670020F0D28E308FFDDFD47F02D206907F979C
:100F7700E520F0C28E907DC6E0F4F58B907DC5E04C
:100F8700F4F58DC28FD28E308FFDDFDFD50CACE547
:0B0F970089540F4430F589C28ED2AFA0
:010FA200222C
:1015A200907DC2E02410547FF50CE030E715907D69
:1015B200C4E0FFAD0C121835901B4EEFF07516719A
:1015C20002187C907DC4E0FF907DC3E0FBAD0C125D
:0615D200000E121B19229D
:10100E00121B19907DC2E0FFC454C0F516E4F535ED
:10101E00E516B44004D2058015E5167004C20580AD
:10102E000DE516B4800575353F800375350FE5382F
:10103E00543F4516F538C204907DC2E030E402D22A
:10104E0004907F97E520F0907DC2E05403F516B42E
:10105E000103121640E516B40203121568E516B424
:06106E000303120DAB228A
:100EC200C2AFE53854CF901B4EF0305904E04410C5
:100ED200F0305707901B4EE04420F0305607901B2D
:100EE2004EE04430F0A204E433901B4FF0907F991F
:100EF200E020E107901B4FE04404F0E50D6007900D
:100F02001B4FE04410F0E5086007901B4FE04420BF
:100F1200F0E50E6007901B4FE04440F0E5096007E2
:100F2200901B4FE04480F0901B50E52FF0D2AF753C
:050F3200169302187C7B
:10152E00907DC2E0F50CE4F516F50C907DC2E0FF5F
:10153E00E50CC39F501874C3250CF582E4347DF579
:10154E0083E0FF1214AC50020516050C80DD901BD3
:0A155E004EE516F07516B102187C78
:0F1AC200121B19C23E907DC2E030E002D23E22DC
:101074001201000100000040970D0101010001026E
:10108400000109022000010100A00009040000027F
:10109400FF0000000705820240000007050202402D
:1010A4000000040309040A035300420049004700F6
:1010B4001E035500530042002D00430041004D0023
:1010C400200045006E00670069006E0065000000A6
:041B270001020408AB
:10052200901B6712110300000000C25DC23BC2545F
:10053200C2401208AF7E107F748E188F19751A1080
:10054200751B86751E10751FA6EE54E07003020619
:1005520086901B6BE4F0A37480F0A3EEF0A3EFF09F
:10056200C374D29FFF74109ECF2402CF3400FEE4E6
:10057200FCFD901B631210F7901B5D12110300002B
:100582000000901B63E0FCA3E0FDA3E0FEA3E0FFFC
:10059200901B5DE0F8A3E0F9A3E0FAA3E0FBC3122D
:1005A20010E6503A901B5FE0FEA3E0FF901B6BE069
:1005B200FCA3E02FF582EC3EF58374CDF0901B5D39
:1005C200E0FCA3E0FDA3E0FEA3E02401FFE43EFE85
:1005D200E43DFDE43CFC901B5D1210F780A4901BEF
:1005E2005D12110300000000901B63E0FCA3E0FD1C
:1005F200A3E0FEA3E0FF901B5DE0F8A3E0F9A3E017
:10060200FAA3E0FBC31210E65049901B5FE0FEA381
:10061200E0FF901B6DE0FCA3E02FF582EC3EF5833A
:10062200E0FD901B6BE0FAA3E02FF582EA3EF58332
:10063200EDF0901B5DE0FCA3E0FDA3E0FEA3E0244F
:1006420001FFE43EFEE43DFDE43CFC901B5D121024
:10065200F78095901B6BE0F518A3E0F519747424EC
:1006620080FF741034FFFE901B61F0A3EFF0C3E52E
:100672001B9FF51BE51A9EF51AC3E51F9FF51FE5A3
:100682001E9EF51ED2E843D820907F95E044C0F02C
:10069200907FAFE04401F0907FAEE0441DF0907F88
:1006A200ADE04404F0D2AF1207372040522040059B
:1006B200D25E121258901B67121103000000007FD5
:1006C200407E927D047C00901B67E0F8A3E0F9A3D2
:1006D200E0FAA3E0FBC31210E650CF2040CC901BFF
:1006E20067E0FCA3E0FDA3E0FEA3E02401FFE43EFB
:1006F200FEE43DFDE43CFC901B671210F780C0E570
:100702008E54F84401F58E304005120302C2403087
:100712005D12C25D1218E2203B07907FD6E020E70F
:10072200F3121956120C47120C47120C47120C47BF
:05073200120C4780D20B
:10030200907FE9E070030203E114700302045524B4
:10031200FE70030204C424FB70030203DB147003A7
:100322000203D51470030203C91470030203CF241D
:10033200056003020513907FEBE024FE6016146053
:100342004224027078E518907FD4F0E519907FD5A9
:10035200F002051A907FEAE0FF1214EDAA06A9073F
:100362007B018B3D8A3E893FEA49600DEE907FD446
:10037200F0EF907FD5F002051A907FB4E04401F0CF
:1003820002051A907FEAE0FF1216D0AA06A9077B9F
:10039200018B3D8A3E893FEA496018EE907FD4F096
:1003A200EF907FD5F0E4907FB5F0907FB47402F0C7
:1003B20002051A907FB4E04401F002051A907FB45E
:1003C200E04401F002051A121ADF02051A121B0597
:1003D20002051A12000302051A121AD102051A9016
:1003E2007FE8E0247F60241460312402705BA23B2A
:1003F200E433FF25E0FFA254E4334F907F00F0E4A2
:10040200A3F0907FB57402F002051AE4907F00F029
:10041200A3F0907FB57402F002051A907FECE0F42D
:100422005480FFC4540FFFE054072F25E024B4F595
:1004320082E4347FF583E05401907F00F0E4A3F07E
:10044200907FB57402F002051A907FB4E04401F087
:1004520002051A907FE8E024FE601D240260030278
:10046200051A907FEAE0B40105C23B02051A907FAB
:10047200B4E04401F002051A907FEAE0703B907FFD
:10048200ECE0F45480FFC4540FFFE054072F25E042
:1004920024B4F582E4347FF583E4F0907FECE054F9
:1004A20080FF131313541FFFE054072F907FD7F0E0
:0304B200E4F5402E
:1004B500E04420F0805F907FB4E04401F0805690E6
:1004C5007FE8E024FE60182402704A907FEAE0B4D9
:1004D5000104D23B803F907FB4E04401F080369028
:1004E5007FEAE07020907FECE0F45480FFC4540F65
:1004F500FFE054072F25E024B4F582E4347FF5832B
:100505007401F08010907FB4E04401F08007907F83
:0C051500B4E04401F0907FB4E04402F038
:0105210022B7
:03003300021B238A
:041B230053D8EF3272
:0D00360000170B0907070605090A0A0CFF51
:10181100052E7E00E52E54032427F582EE341BF5B8
:1018210083E493FFE52454F0FEEF4EF5249080030A
:04183100E524F02298
:100DAB00753503C249D227908003E524F0E4F5168C
:100DBB00F536752FFF7D64E516C3947050481218F5
:100DCB001185140CC3E514950CC39D40F77D05E507
:100DDB00366013FF0536EFC3940340DBE52E20E0AE
:100DEB00D6752F098020908000E0139259AF16051D
:100DFB0016EFC3940C40083044053059020536A257
:100E0B0059B3924480B1532EFED259C244C257C239
:100E1B00567536FFD249C227908003E524F0E5369C
:0D0E2B0070FCE4F535D205907F97E520F0CE
:010E38002297
:10164000C249305604D25A8026C25A305921D25744
:10165000C259E52E5403901B2793FFE52454F0FE56
:10166000EF4EF524908003E524F0E4F536F537D20B
:0216700049220D
:10156800C249305704D24D802EC24D304429D2563C
:10157800C244C207907F97E520F0E52E5403901BE4
:101588002793FFE52454F0FEEF4EF524908003E501
:0A15980024F0E4F536F537D24922BD
:03000B00020046AA
:10004600C0E0C0F0C083C082C0D075D000C000C080
:0D00560001C002C003C004C005C006C00701
:10006300901B42E004F0E0540760030202C72049FA
:100073000302012F20570620560302011F20560FAB
:10008300E537700B901B44E06409600302012FE520
:10009300367071908000E0139245E5377005750F57
:1000A300FF801C302719A245304201B3501130574D
:1000B3000830420B85370F800620420385370FC275
:1000C30027A24592421218110537E537900036935F
:1000D300F536E537640C7054908003E524F0850F02
:1000E3002F305714D244C257D207907F97E520F0A0
:1000F300304D391215688034D259C256305A2D12F8
:10010300164080281536E536B40121E537C3940738
:10011300401AD227908003E524F08010E536600C66
:10012300D536095324F0908003E524F0303E75C2A0
:100133002E908004E525F09080027401F0741DF088
:100143007419F09080007474F0908001747FF075DE
:100153003D04908000748FF09080017441F0908092
:10016300027419F0D53DEB753D04908001E4F090E5
:1001730080027410F0D53DF29080007474F090808A
:1001830001747FF09080027401F0908000E521F00B
:10019300908001E522F0908002E523F0D22E90803A
:1001A30004E525F0305117303C07C23C121A3E805B
:1001B3000DAF171517EF7006C251D2468063901B1F
:1001C30044E004F0E0640A60030202C7F00514E5AA
:1001D300147006901B45E004F0D25020460302023F
:1001E30073E5385403FFBF01082059033044020567
:1001F30038E5385403FFBF021DAF171517EF70160C
:10020300AF111511EF700FAF0B150BEF7008304FD7
:10021300101215680538E5385403FFBF030E305933
:100223000B304E05C2431211345338FCE538540CDD
:10023300FFBF040C20440330590674042538F538F5
:10024300E538540CFFBF081AAF3C153CEF7013AFF1
:10025300391539EF700C304C1412156874042538B5
:10026300F538E538540CFFBF0C063059035338F307
:10027300305306E514540F7035753D00E50D6005E8
:10028300433D01150DE5086005433D021508E50EE4
:100293006005433D04150EE5096005433D08150956
:1002A300E52054F0453DF520907F97E520F0E535B6
:1002B300600655147002B205907F97E520F0E514AF
:1002C300543F600330581D30431AB208B20990807E
:1002D30000E521F0753D04D53DFDB208B2099080DB
:0402E30000E521F021
:1002E700D007D006D005D004D003D002D001D0006B
:0B02F700D0D0D082D083D0F0D0E03215
:101AB200040103000505000301000200FFFFFEFE12
:1008AF00D23B907F92E054FDF0E4907FE2F0F5862A
:1008BF00907F9574C3F0907F9E74FBF0907F93743C
:1008CF0028F0E4907F94F0907F9C747DF0907F9659
:1008DF007401F0907F9D74FFF0907F977430F090CB
:1008EF007FDD7409F0907FA1E04401F0907FB27436
:1008FF0000F0A37446F0907FAFE04406F0758C06CD
:10090F00E58954F84402F589538EF7D28CD2A97534
:10091F002460908003E524F0AF3A1216A3D206901C
:10092F007F97E520F0753840D24675230175217405
:10093F0075227F752503908000E521F0908001E5F9
:10094F0022F0908002E523F0908004E525F090805E
:10095F0010E526F0901B487401F07D0C7F401214B7
:10096F006AE4FD7F7012146A7DD8E4FF12146A7D69
:10097F00407F1012146AD24A7D0C7F2012146A7DB8
:10098F001E7F5012146A7D1E7F3012146AE4FD7FA1
:04099F006002146A74
:10073700908006E4F0A3740AF0908008E4F0A374B4
:1007470009F090800AE4F0A304F0D22E908004E52B
:1007570025F0D22FE525F085140C908000E030E1DC
:100767000AC3E514950CD3940A40EF121AED120D43
:10077700AB7F01121672753304E4901B49F0A3F0A6
:10078700750C02E50C2410FD7FA0121835901B4A4A
:10079700E02FF0901B49E03400F0050CE50CC39402
:1007A7002040E07D117FA0121835EFFE901B4AE034
:1007B7002400F0901B49E03EF07D107FA012183511
:1007C700901B4AE02FF0901B49E03400F0E0F470F2
:1007D70003A3E0F4702F7D137FA01218358F337DAC
:1007E700167FA01218358F0D7D1A7FA01218358F2E
:1007F7000E7D247FA01218358F0CE50C139238E577
:100807000CA2E2924BE53324FB601524FB6016240F
:10081700FE6017146021146023800075301880254E
:100827007530308020753010801B753046D22D9082
:100837008004E525F0800E7530208009753034D2AC
:100847003AD208D243E50C30E50A901B5C746FF08E
:10085700D2558008121423901B5CEFF0E4F50CE5E9
:100867000EC394804003750C01E50C2450FFE50E80
:1008770025E0FD12146AE4F50CE50DC394804003EE
:10088700750C01E50C2460FFE50D25E0FD12146AE7
:10089700E4F50EF50DA238922A908004E525F0D2F2
:0808A70004907F97E520F02288
:100B73001214238F15205503020C1BE4FD901B5CFC
:100B8300E0FCC3951540027DFFE514547FFFBF04CD
:100B930017ED600C901B43E0F4600DE004F0800857
:100BA300901B43E0600214F0E5145407707CED6081
:100BB30030ECC39515F53EE49400F53DE53EAE3DBE
:100BC3007803C333CE33CED8F9F53E8E3D901B4325
:100BD300E0FB7E00253EEE353D7039EB253EFD8082
:100BE30033ECFFE515C39FF53EE49400F53DE53E88
:100BF300AE3D7803C333CE33CED8F9F53E8E3D9068
:100C03001B43E0FFFBC3E53E9BE53D94005005C35A
:100C1300EF953EFD8D108012901B43E0600CE514B0
:100C230054077006E51060021510E510D3953A409D
:100C330002053AE510C3953A5002153AAF3A121637
:030C4300A3C250F9
:010C4600228B
:100C4700305C3F907DC0E0F50CA3E0FFC4540FF586
:100C570016E50CB4A509E516901AB293B4FF051270
:100C6700193B801CE516901AB293FF907DC1E054A2
:100C77000F6F6004EFB4FE05120E398003121B1EBE
:100C8700C25C30522FE534702BC3E52D951DE52C42
:100C9700951C5011E52DAE2C7805CEC313CE13D875
:100CA700F9F534800FE51DAE1C7805CEC313CE13BE
:100CB700D8F9F534538EF8120A92058E30480F1280
:100CC70009A3A24792475021C248C247801BE50AA1
:100CD7006017E51D2513FFE51C3512FED3EF9400C1
:100CE700EE94105004D248150A305006205B0312C8
:100CF7000B73E5385403FFBF0210E511D39400507E
:0D0D070006E50B94004003C25822D258228A
:08000300907FEAE0F544D322EE
:0E1AD100907F00E544F0907FB57401F0D322C1
:081B0500907FEAE0F543D322D2
:0E1ADF00907F00E543F0907FB57401F0D322B4
:10198800C0E0C083C082D2405391EF907FAB740116
:08199800F0D082D083D0E032D0
:1019D000C0E0C083C0825391EF907FAB7404F0D01D
:0619E00082D083D0E0324A
:1019E600C0E0C083C0825391EF907FAB7402F0D009
:0619F60082D083D0E03234
:1019FC00C0E0C083C0825391EF907FAB7410F0D0E5
:061A0C0082D083D0E0321D
:1019A000C0E0C083C082D25D5391EF907FAB7408DA
:0819B000F0D082D083D0E032B8
:1019B800C0E0C083C082D25C5391EF907FAA7404C8
:0819C800F0D082D083D0E032A0
:100A9200907FB8E020E114E53460081534792078BD
:100AA200208026E52D7005E52C7001227820E52DA9
:100AB200C398E52C94005002A82DE8F9305270E555
:100AC2001DC398E51C940040E2907FE27450F074DC
:100AD20000907FE4F0747E907FE3F0907FE57420D5
:100AE20098702C7802C2AFF0F0F0F0F0F0F0F0F075
:100AF200F0F0F0F0F0F0F0F0F0F0F0F0F0F0F0F0F4
:100B0200F0F0F0F0F0F0F0D8DED2AF8008C2AFF033
:100B1200F0D8FCD2AF907FE27400F0907FB9E9295F
:100B2200F0C3E51D99F51DE51C9400F51C802F8589
:100B320032848531857400907FE4F0747E907FE387
:100B4200F0907FE5C2AF0586E0A30586F00586E05A
:100B5200A30586F0D8F0D2AF907FB9E929F0858459
:100B620032858531E52DC399F52DE52C9400F52CC0
:010B72002260
:011B2D003285
:1009A300E53B24F97003020A5D24076003020A9100
:1009B300204803020A91C2AFC22F908004E525F0BC
:1009C3007F05121B2BC22E908004E525F0304A1FB1
:1009D300303A12C243304E03121A3E901B48E0FFD6
:1009E300121A53801F901B48E0FF12192080153004
:1009F300380A901B48E0FF121A128008901B48E047
:100A0300FF121903901B49E0FEA3E0FF8E45F54654
:100A1300901B46E0FCA3E0FDEF2DFBEE3CCB251342
:100A2300F546EB3512F545908006F0A3E546F0C395
:100A33009FF546E5459EF545908008F0A3E546F011
:100A430090800AECF0A3EDF0D22E908004E525F01F
:100A5300D22FE525F0D2AF753B07908000E020E16F
:100A63002DE513251DF51DE512351CF51CE50A6062
:100A730018E51D2513FFE51C3512FED3EF9400EE98
:0E0A830094105005150A0209B9E4F53BD2475C
:010A91002242
:101A6800C3907FA57800E020E003D8FA2220E2FCAA
:051A780030E1F9D3226A
:1018C000C2AF907FA57480F0907FA6EF54FEF01217
:1018D0001A68500D7400F0907FA6EDF0121A68504F
:0218E0000022E4
:10000E001218C05009907FA6EBF0121A68C3907FA9
:10001E00A57440F05008907FA6E0FF907FA5E020E9
:05002E00E6FCD2AF2248
:101835001218C0501B7480F0907FA6EF54FE44012F
:10184500F0121A68500A7420F0907FA6E0121A6808
:04185500D302001C9E
:101A1200908001E522C2E4F06403C2E4F0D2E4F073
:061A2200DFF8E522F022CE
:1017C800EF2E601DD3121970908001E5220E641867
:1017D800F06403F06418F06403F0DFF2DEF0E52251
:0517E800F0C3021970BE
:101A2800908002E523D2E3F07805121B0DC2E3F0A3
:061A380012160CC23D2253
:10160C00908001E5227D7D7C0B7B10C2AF6BF06C72
:10161C00F06BF06CF06BF06CF06BF06CF06BF06CE2
:10162C00F06BF06CF06BF06CF06BF06CF0DDDED20C
:04163C00AFD23D22CA
:10177900EE2F6020D3121970908001E5220EC2E588
:10178900F0C2E3F06403F0D2E3F06403F0DFF2DEC9
:08179900F0E522F0C302197013
:10190300908001E522C2E5F0C2E3F06403F030E326
:0D19130003C2E3F0D2E3F0DFF5E522F0229D
:10195600907FD6E030E712E04401F07F147E00125B
:0A19660011E9907FD6E054FEF02254
:1018E200907FD6E04480F043870100000000002290
:07125800907FD6E04408F08E
:03125F00E4F53D76
:04126200E054FBF069
:03126600E4F53D6F
:10126900E04408F0305E04E04402F07FDC7E0512C1
:1012790011E9907F92E030E3077FDC7E051211E9E6
:10128900907FAB74FFF0907FA9F0907FAAF0539103
:08129900EF907FD6E054F7F05E
:0312A100E4F53D34
:0512A400E04404F0220B
:0216D000A90768
:1016D200AE1EAF1F8F828E83A3E064037017AD012D
:1016E20019ED7001228F828E83E07C002FFDEC3E8B
:0916F200FEAF0580DF7E007F00E1
:0116FB0022CC
:0214ED00AD0749
:1014EF00E4FCAE1AAF1B8F828E83A3E06402702AD6
:1014FF00AB040CEBB50501228F828E83A3A3E0FA18
:10150F00A3E08A41F5426241E5416242E542624110
:0E151F002FFBE5413EFEAF0380CC7E007F0037
:01152D00229B
:1011E9008E3E8F3FE53F153FAE3E7002153E4E6085
:0711F900051218F280EE223E
:1018F2007400F58690FDA57C05A3E582458370F909
:0119020022C2
:03004300021200A6
:10120000021988000219E6000219D0000219A00094
:101210000219FC00021B2D00021B2D00021B2D00D9
:10122000021B2D00021B2D00021B2D000219B8000D
:10123000021B2D00021B2D00021B2D00021B2D0086
:10124000021B2D00021B2D00021B2D00021B2D0076
:08125000021B2D00021B2D0002
:03000000021AF9E8
:0C1AF900787FE4F6D8FD758146020522D6
:1010D400EF8DF0A4A8F0CF8CF0A428CE8DF0A42E30
:0210E400FE22EA
:1010E600EB9FF5F0EA9E42F0E99D42F0E89C45F060
:0110F60022D7
:0C10F700ECF0A3EDF0A3EEF0A3EFF0226C
:10110300A8828583F0D083D08212111A12111A1289
:10111300111A12111AE473E493A3C583C5F0C583AE
:10112300C8C582C8F0A3C583C5F0C583C8C582C836
:011133002299
:00000001FF
